:100000000C949E020C94AE130C9487130C94C602AD
:100010000C94C6020C94C6020C94C6020C94C60240
:100020000C94C6020C94C6020C94C6020C94310FB8
:100030000C94C6020C94C6020C94C6020C94C60220
:100040000C943D130C94C6020C9430120C940A12BA
:100050000C94C6020C94C6020C94C6020C94C60200
:100060000C94C6020C94C6029109AA092F0A300BFF
:10007000540B750B810B230B4E414E494E4954597D
:10008000494E46CDCCCC3D0AD7233C17B7D1387763
:10009000CC2B329595E6241FB14F0A000020410079
:1000A00000C84200401C4620BCBE4CCA1B0E5AAEC3
:1000B000C59D7400407A10F35A00A0724E180900D2
:1000C00010A5D4E80000E87648170000E40B5402BD
:1000D0000000CA9A3B000000E1F5050000809698F8
:1000E00000000040420F000000A086010000001048
:1000F0002700000000E8030000000064000000008A
:10010000000A00000000000100000000002C76D86A
:1001100088DC674F0823DFC1DFAE59E1B1B796E550
:10012000E3E453C63AE651997696E8E6C28426EBB4
:10013000898C9B62ED407C6FFCEFBC9C9F40F2BAC7
:10014000A56FA5F490055A2AF75C936B6CF9676D5F
:10015000C11BFCE0E40D47FEF520E6B500D0ED90B4
:100160002E0300943577050080841E080000204E81
:100170000A000000C80C333333330F986E1283111A
:1001800041EF8D2114893BE65516CFFEE6DB18D1F1
:10019000844B381BF77C1D901DA4BBE424203284C3
:1001A000725E228100C9F124ECA1E53D273D005398
:1001B00061766520696E20454550524F4D00290AF1
:1001C0000020002028004672656520284229202052
:1001D0003A20002D2D2D005057443D005553523DDF
:1001E000004349443D005356523D004D534B3D00A2
:1001F0004757593D00444E533D0049503D20004D66
:1002000041433D004856433D004641433D0057446D
:10021000473D002D2D2D000A55534147453A0A20F0
:10022000204641433D7878782E78202028474D207D
:100230007475626520666163746F72290A202048B4
:10024000564C3D787878205B302D3235355D20284E
:100250004869676820566F6C7461676520636F6ECC
:1002600076657273696F6E290A202052535420619B
:100270006C6C20636F756E746572730A0A20204D72
:1002800041433D48483A48483A48483A48483A483D
:10029000483A4848202868657861290A2020495052
:1002A000203D7878782E7878782E7878782E78783F
:1002B000780A2020444E533D7878782E7878782E2E
:1002C0007878782E7878780A20204757593D7878C2
:1002D000782E7878782E7878782E7878780A20209A
:1002E0004D534B3D7878782E7878782E7878782E24
:1002F0007878780A20205356523D7878782E78788E
:10030000782E7878782E7878780A20204349443DF2
:100310003C636C69656E742069643E2028352063F7
:1003200068617273206D61782E290A20205553521E
:100330003D3C6E616D653E202838206368617273B4
:10034000206D61782E290A20205057443D3C706171
:1003500073733E202838206368617273206D617862
:100360002E290A0A20205744473D5B302C315D205E
:100370005761746368646F670A20204F5054494F77
:100380004E5320202053686F7720636F6D6D616E30
:100390006473202620706172616D657465727320CC
:1003A00076616C7565730A202053415645202020E4
:1003B0002020205361766520706172616D657465DF
:1003C000727320696E746F20454550524F4D0A205C
:1003D000204D454D4F52592020202053686F7720E3
:1003E00066726565206D656D6F72790A20205645CD
:1003F0005253494F4E20202053686F772066697210
:100400006D776172652076657273696F6E0A0A4B4B
:1004100065657020627574746F6E206465707265B6
:100420007373656420647572696E6720737461729A
:1004300074757020746F2064697361626C65206EDE
:100440006574776F726B20616E64206561736520DF
:10045000636F6E66696775726174696F6E20746828
:10046000726F756768205553422E0A000000000025
:10047000240027002A0000000000250028002B008F
:1004800000000000230026002900040404040404E2
:100490000404020202020202030303030303010233
:1004A0000408102040800102040810200102040802
:1004B00010200000000800020100000304070000F3
:1004C0000000000000005374617469632049503AD1
:1004D00020003E3E20434F4E46206D6F6465003E37
:1004E0003E204D515454206D6F6465002062792088
:1004F00041644E6F766561202D203230313928639A
:100500002900432D474D204D515454207600204161
:1005100056473D00204856563D0020454C503D0072
:10052000204156473D0020544F543D00204D415836
:100530003D0020434D503D002F009A2811241FBE3E
:10054000CFEFD8E0DEBFCDBF11E0A0E0B1E0EAE43C
:10055000F5E602C005900D92A63DB107D9F727E058
:10056000A6EDB1E001C01D92A230B207E1F712E0A2
:10057000CEE9D2E004C02197FE010E945332CD396A
:10058000D107C9F70E94FA220C94A3320C94000000
:10059000FC01448555854115510551F0FB01248529
:1005A00035852115310521F081E04217530709F007
:1005B00080E00895DC011C96ED91FC911D97309729
:1005C00039F08181811106C0808182958170089502
:1005D00080E0089581E0089580E090E00895DC01D6
:1005E000ED91FC91028CF38DE02D099591E0892726
:1005F0000895089580E090E00895E091D601F0E03C
:10060000EE0FFF1FE952FE4F808191810196918389
:1006100080838091DC029091DD02A091DE02B09196
:10062000DF020196A11DB11D8093DC029093DD02D3
:10063000A093DE02B093DF0281E08093E50208958B
:10064000FC01848595850C94B720CF93DF931F928E
:10065000CDB7DEB7698341E050E0BE016F5F7F4FE9
:10066000FC01848595850E94B7200F90DF91CF9182
:100670000895CF93DF93EC010E94061DEC85FD8564
:10068000309739F0808186FF06C081E09181911119
:1006900003C080E001C081E0DF91CF910895EF9227
:1006A000FF920F931F93CF93DF938C017B01EA019D
:1006B000DC01ED91FC910488F589E02D0995F701A5
:1006C000828190E0982F88272381822B9827892781
:1006D0009827248130E0322F22274581242B32278E
:1006E000232732277C2F6D2F40918A0350918B0353
:1006F0004F5F5F4F4115FDE75F0710F040E050E1AD
:10070000D42FC52FECE8F3E0A0E0A43059F0B18D70
:10071000BB2329F0E480F580EC16FD0649F3AF5FBA
:100720007E96F3CF50938B0340938A0310920C0470
:1007300040E0C0E0D0E0AEE14430C1F0A49FF00161
:100740001124E457FC4F518D511104C040930C0407
:10075000EF010EC0573031F4209729F0B28D5A8D39
:100760005B1708F0FE014F5FEF01E6CF40930C04EA
:10077000209719F480E090E040C042E0498F40911A
:100780005E024C8740915F024D87409160024E8728
:10079000409161024F8740E052E05B8B4A8B5D8B5A
:1007A0004C8B41E050E0598B488B1B8E4A8F43E0C5
:1007B000488F1E8A40E14F8B40918A0350918B03F2
:1007C0005427452754275D834C837F836E83998309
:1007D00088833B832A83898D8F7061F20E94061D76
:1007E000898D8F708330B9F78C8D9D8DD8011D96C2
:1007F0009C938E931C9781E090E0DF91CF911F91A5
:100800000F91FF90EF900895CF93DF93EC018C85CB
:100810009D85009781F0FC012081222361F00196E3
:100820000E943D1FEC85FD85908196FF02C01082DD
:1008300002C0906290831D861C86DF91CF910C943C
:10084000061DEF92FF920F931F93CF93DF9300D07B
:10085000CDB7DEB77C018B0149835A830E943113E7
:10086000F701E857FF4F6083718382839383D70139
:1008700014968D919C911597DC01ED91FC9102806D
:10088000F381E02D49815A81B8010F900F90DF91DB
:10089000CF911F910F91FF90EF9009941F93CF93E9
:1008A000DF93EC01162F0E943113FE01E857FF4F32
:1008B00060837183828393838C819D81DC01ED91C0
:1008C000FC910190F081E02D612FDF91CF911F917C
:1008D0000994EF92FF920F931F93CF93DF939C01A4
:1008E000FB011092890390E08BE0983031F1899FF1
:1008F00070011124E701CF5CDC4F688179816115BB
:100900007105C9F04A815B8141155105A1F0D901FA
:100910000D911C9111970617170769F412966D91A6
:100920007C9113976417750731F490938903D7016D
:10093000AB5CBC4F2AC09F5FD8CF90E08BE0983073
:1009400091F0899FE0011124CF5CDC4F48815981EF
:10095000452B39F44A815B81452B19F49093890327
:100960000AC09F5FECCF1092590210925802109269
:100970008903C1E3D3E0D9014D915D916D917C91E3
:10098000DE014D935D936D937D9386E001900D9212
:100990008A95E1F71A86DF91CF911F910F91FF9011
:1009A000EF900895CF93DF9300D000D000D0CDB763
:1009B000DEB780918502909186028F3F2FEF9207DC
:1009C00059F420918702309188022F3F3F4F21F444
:1009D00086E0E7E0F1E0F3C020912D0330912E0393
:1009E00028273927409125035091260324233523B6
:1009F000232B91F4609187027091880220912F033C
:100A00003091300326273727409127035091280340
:100A100024233523232B89F08091290390912A03E5
:100A200090935B0280935A0280912B0390912C0348
:100A300090935D0280935C0208C090935B02809368
:100A40005A0270935D0260935C0220915A023091C9
:100A50005B0240915C0250915D0280E09BE0883037
:100A6000B9F1989FD0011124AF5CBC4F6D917C917E
:100A700011972617370751F512966D917C911397B0
:100A80004617570719F5FD01349614966C91149783
:100A9000611118C015966C911597611113C01696C7
:100AA0006C91169761110EC017966C911797611192
:100AB00009C018966C911897611104C019966C9131
:100AC000662321F08093890386E079C08F5FC7CFCA
:100AD0008093890346E050E06FEF70E087E692E094
:100AE0000E94813286E0E7E8F2E0DF01282F1D92C4
:100AF0002A95E9F7E2EEF4E0ADE6B2E0982F019036
:100B00000D929A95E1F7E2EEF4E0ADE7B2E0982FAE
:100B100001900D929A95E1F720915A0230915B0273
:100B200030938E0220938D0220915C0230915D0201
:100B30003093900220938F0220912D0330912E0349
:100B4000309384022093830220912F03309130034D
:100B5000309386022093850220E031E030937C02BE
:100B600020937B02309376022093750228E030E0D8
:100B700030937802209377028093790294E09093E7
:100B80007A0228E036E030937402209373022DE954
:100B900032E03093B1062093B0062AE230E0309381
:100BA000630220936202BE016F5F7F4FDB011D92E3
:100BB0008A95E9F78AE592E00E9469041EC0A7E6DB
:100BC000B2E001900D928A95E1F786E0E2EEF4E062
:100BD000ADE6B2E001900D928A95E1F788E090E0F1
:100BE00090937402809373028091620290916302E9
:100BF0000E96909363028093620226960FB6F89445
:100C0000DEBF0FBECDBFDF91CF910895FF920F934E
:100C10001F93CF93DF93C091B306D091B4062DE913
:100C200032E03093B1062093B0063093AD062093A6
:100C3000AC06833059F4898D8F70833009F0FBC581
:100C400088899989892B09F0F6C57EC0823009F020
:100C50007FC0809161028F5F80936102811113C018
:100C6000809160028F5F8093600281110CC080913F
:100C70005F028F5F80935F02811105C080915E02E9
:100C80008F5F80935E021092630210926202109254
:100C9000AF061092AE06898D982F9D7F953041F456
:100CA0008A8D8F5F8A8F883709F0C5C5198EC3C5B5
:100CB000882309F4C0C528893989232B09F440C049
:100CC0009A8D2FEF290F2A8F9111B5C59B8D9830E2
:100CD00031F02FEF280F223048F4953039F4198E77
:100CE00080E88093B2060E94671F51C4953038F4A3
:100CF00023E0092E01C0220F0A94EAF701C020E385
:100D00002A8F9F5F9B8F8F708330A1F048F48130D2
:100D100009F42BC2823009F08EC51092960228C2C7
:100D2000863009F443C4883009F440C4843009F0A3
:100D300082C53CC484E08093B2060E94671F5CC4F5
:100D40008F70833009F077C588E08093B20614C4B1
:100D500080917502853409F06EC58091770290E02C
:100D6000982F882720917802820F911D209162028E
:100D7000309163022817390708F45DC59093630228
:100D80008093620280917B028F7309F054C5F090CA
:100D90007C02F11050C5C0912D03D0912E032097F5
:100DA00031F480912F0390913003892BA1F0809131
:100DB0008502909186028C179D0709F03CC5209111
:100DC00087023091880280912F0390913003281779
:100DD000390709F030C50E945B17019609F02BC551
:100DE00080917E028630B1F1813009F024C5809176
:100DF0008902883009F01FC51092890280918B0208
:100E000090918C02873F4FEF940710F0099601C034
:100E1000089690938C0280938B028091810290912E
:100E20008202909386028093850280918302909142
:100E300084029093880280938702D0938202C093A9
:100E4000810280912F0390913003909384028093CC
:100E50008302F5C40E94D616019609F0ECC42091D5
:100E60008B0230918C028091890290918A0260916C
:100E7000810270918202E0918302F09184020CE879
:100E800013E0D80159964C9159974423C1F0149618
:100E90000D90BC91A02D2A173B0789F4E801AE8183
:100EA000BF818A179B0759F4A881B9816A177B070C
:100EB00031F4AA81BB81EA17FB0709F470C1025E15
:100EC0001F4FD4E004301D07E1F6809196028F7326
:100ED0008230E1F4309357022093560280E0843050
:100EE00099F0E82FF0E0EE0FFF1FEC5FFB4F408121
:100EF00051818F5F2417350791F710920C0480E021
:100F0000C0E0D0E09EE17CC080930C04809196020A
:100F100082FD91C484E18093960288E290E09093F0
:100F200063028093620280E5809395023091900283
:100F3000809194028093900220918F02809193027D
:100F400080938F022093930290918E02809192025F
:100F500080938E029093920280918D0280930C0474
:100F60004091910240938D02809391023F5F3093B4
:100F7000940231110DC02F5F20939302211108C0FC
:100F80009F5F90939202911103C08F5F80939102B3
:100F90008091890290918A02909357028093560221
:100FA00020918B0230918C0230938A022093890227
:100FB00090938C0280938B028091810290918202A7
:100FC000909386028093850280918302909184029F
:100FD000909388028093870280912D0390912E0335
:100FE000909382028093810280912F03909130032D
:100FF0009093840280938302E0C3473099F08F5F1F
:101000008430F1F0282F30E0929FF001939FF00D93
:101010001124E457FC4F418D4111EFCF80930C0414
:10102000EF0110C0209721F0528D4A8D451738F7F7
:10103000929FE001939FD00D1124C457DC4FDFCF66
:1010400080930C04209709F4F6C3D093B406C093A0
:10105000B30683E08A8F888F1E8A84E08F8B1B8E75
:1010600080918B0290918C029D838C838091890268
:1010700090918A029F838E83809181029091820257
:101080009983888380918302909184029B838A83D1
:1010900081E0898F80915E028C8780915F028D87CD
:1010A000809160028E87809161028F8781E090E05D
:1010B000998B888B809190028B8780918F028A8791
:1010C00080918E02898780918D02888781E090E0EF
:1010D0000E94DD2280919502982F907F913508F42F
:1010E00044C082958F7090E00597880F991F880FF4
:1010F000991F20915502EF2DF0E0E817F9078CF5C4
:10110000E959FD4F26A9211105C0F0920C04109257
:1011100055022BC0213011F4F394EDCF2230E1F4CD
:1011200037A93430C9F4F0920C042093550280ADF5
:1011300090E0982F882721AD822B909357028093BF
:1011400056028130E2E09E0710F080E092E09B8B37
:101150008A8B9D8B8C8B09C037A9332311F0F30E3A
:10116000CACFF0920C042093550280E1809396023E
:101170008091960282608093960282E080939D0225
:1011800094E090939E0280939F021092A0028CE2C2
:1011900090E0909363028093620280E6BCC2E80113
:1011A0001093B4060093B3061092B20630919602E3
:1011B000F32FF470FF2E32FF03C0198E80E24BC272
:1011C0002091950222952F70220F220F20930C045C
:1011D00080916202909163024497821B91099093DF
:1011E0006302809362024F70423021F4232F2F73E9
:1011F000223109F1892B19F4832F8370E1F090914A
:101200008D02D80118968C91189798137AC29091F4
:101210008E0219968C911997981373C290918F0230
:101220001A968C911A9798136CC2909190021B9603
:101230008C91981366C234FF63C0F801608971898C
:101240006115710509F45CC0C8010C960E94A722C3
:101250003091910280915102381352C02091920234
:101260008091520228134CC09091930280915302B6
:10127000981346C08091940240915402841340C058
:10128000D8011C963C931C971D962C931D971E9677
:101290009C931E971F968C931F975B968C915B97E0
:1012A000811126C056969C91569758968C915897C6
:1012B0005A962C915A97821B292F2695269526956A
:1012C000821B980F56969C93569787FD819557964B
:1012D0002C915797322F36953695231B820F5796B0
:1012E0008C935797969596959695890F58968C93CB
:1012F00081E08093B206F801808D828F118A108A76
:10130000D80159962C91E22FEF708E2F90E0FC01BE
:101310003197E830F10508F08EC2EC5CFF4F0C9479
:1013200053328091B20680FF86C283E0F801818F3C
:1013300080E48093B206118A108A809162029091B3
:101340006302009709F414C122E42093B2060E94BC
:10135000DD220EC18091B20680FF76C08091960298
:101360008F73823109F070C080919502982F907F21
:10137000913508F449C082958F7090E00597880FE9
:10138000991F880F991F20915502EF2DF0E0E81763
:10139000F907B4F5E959FD4F26A9211105C0F092CE
:1013A0000C041092550230C0213011F4F394EDCFAB
:1013B000223009F537A93430F1F4F0920C0420936F
:1013C000550280AD90E0982F882721AD822B909315
:1013D0005702809356028130F2E09F0710F080E0C0
:1013E00092E0D80153969C938E93529755969C9376
:1013F0008E93549709C037A9332311F0F30EC5CF4C
:10140000F0920C042093550283E0F801818F8091C3
:101410008D02808780918E02818780918F028287E2
:1014200080919002838781E090E00E94DD2282E437
:101430008093B206D80151961C921E92509710923A
:1014400063021092620294C080E28093B2060E940E
:10145000671FE091B306F091B406118E57CD8091CD
:10146000960280FF2EC024FD2CC0F801808991894E
:10147000892B09F0E0C1809162029091630201968C
:101480000E94DD228091B206982F90619093B2065F
:101490002091620230916302232B19F082618093C4
:1014A000B2060E94671F81E090E0D80151969C939C
:1014B0008E93509788E059968C9359975B961C921F
:1014C00075C085FF1DC080919B0290E0982F8827F2
:1014D00030919C02832B4091B0065091B106480F89
:1014E000591F5093B1064093B0064091620250914B
:1014F0006302FA01E81BF90BF0936302E0936202C6
:1015000040916202509163024115510551F024FD52
:1015100008C09091B20692609093B206CA010E94F0
:10152000DD228091970290E0982F882720919802E1
:10153000820F911D9093570280935602D8015496C2
:101540002D913C9155972817390710F0892B21F4DC
:101550003093570220935602809156029091570281
:10156000F801938B828B8091B206837009F463C17A
:101570001092AF061092AE060E94671F8091B206CD
:1015800085FF07C01092AF061092AE06198E84E157
:10159000B9C084FF0DC01092AF061092AE0681E074
:1015A00090E0998B888B84E0898F1B8E81E1AAC0A3
:1015B0002091AE063091AF0621153105E1F080FF94
:1015C00002C0198A188A88899989009781F48A89C2
:1015D0009B898217930720F49093AF068093AE0601
:1015E0008091AE069091AF06998B888B04C0909342
:1015F000AF068093AE061B8E8091AC069091AD062F
:101600009093B1068093B0068091AE069091AF069C
:10161000892B59F088899989009739F08896909399
:1016200063028093620288E10BC08091B20681FF61
:1016300002C188E290E0909363028093620280E1AD
:101640008093960267C08091B20680FFF4C0D801F3
:1016500059961C9280E18093B2060E94671FEBC0EE
:101660008091620290916302009711F00E94DD2246
:10167000909196028091B20690FF0EC080FF07C045
:1016800087E0F801818F128E118A108A1DC086E0D2
:10169000D80159968C9318C080FF20C085E0E801DE
:1016A000898F198A188AC7C080916202909163025B
:1016B000009711F00E94DD228091960280FF0EC0FB
:1016C00087E0F801818F128E81E090E00E94DD2298
:1016D00080E18093B2060E94671F13C0809162026E
:1016E00090916302892B69F4A6C08091B20680FFB5
:1016F000A2C087E0D80159968C9359975A961C92AC
:101700009AC080E18093960288E290E09093630211
:101710008093620280E58093950288858093910290
:101720008985809392028A85809393028B8580932A
:1017300094028C8580938D028D8580938E028E8598
:1017400080938F028F858093900286E080937E0243
:101750008C819D8190938A02809389028E819F81E2
:1017600090938C0280938B0280912D0390912E0395
:10177000909382028093810280912F039091300395
:10178000909384028093830288819981909386024A
:10179000809385028A819B8190938802809387023F
:1017A000898D84FF05C0109298021092970205C09F
:1017B00082E0809397021092980280E480937D02E9
:1017C00080916202909163029093770280937802F5
:1017D00010929C0210929B0210929A02109299020F
:1017E0000E94D6168095909590939A0280939902C4
:1017F00085E4809375021092760210927C0210921A
:101800007B0280914F02909150020196909350027A
:1018100080934F029093790280937A021092800213
:1018200010927F020E945B178095909590938002A2
:1018300080937F0204C010926302109262021092A1
:10184000B206DF91CF911F910F91FF9008951092F2
:10185000E3021092E2021092D8021092D902109282
:10186000DA021092DB021092DC021092DD0210927A
:10187000DE021092DF021092E1021092E00288E78D
:10188000E7EDF1E0DF011D928A95E9F71092D601AC
:101890001092D4021092D5021092D6021092D70262
:1018A00008958F929F92AF92BF92CF92DF92EF9264
:1018B000FF920F931F93CF93DF93CDB7DEB76C9753
:1018C0000FB6F894DEBF0FBECDBF9C8F8B8FAE01DD
:1018D000455E5F4F67E671E00E94042B7E0123E1C5
:1018E000E20EF11CBC01C7010E949C328701F70186
:1018F00001900020E9F73197EE19FF09C8018E1910
:101900009F098E179F0758F4F8018081082E000C5C
:10191000990B0E945E32F80181938F01E8CF1B89F9
:101920001F3319F487E192E025C2173551F4EB8D8E
:10193000FC8D81E09081913309F080E080938B05EC
:1019400078C2163469F48B8D9C8D0E94D42A6093E2
:10195000C9057093CA058093CB059093CC0569C2E5
:10196000183439F48B8D9C8D0E94D82A8093C80539
:1019700060C269E671E0C7010E949332892B39F495
:101980000E94270C109285001092840052C21D34D0
:1019900021F58C898134E1F56B8D7C8DCE0101962A
:1019A0000E949C326DE671E0CE0101960E94FF2AF2
:1019B0000CE815E0009709F43CC240E150E060E01B
:1019C00070E00E94C229F80161938F016DE671E019
:1019D00080E090E00E94FF2AEDCF193429F46B8D4E
:1019E0007C8D82E995E00AC0143459F48C898E34D8
:1019F00009F0D9C16B8D7C8D88E995E00E94D711E3
:101A000018C2173469F46B8D7C8D8EE995E0F6CFA2
:101A1000833509F0B2C16B8D7C8D84EA95E0EECF01
:101A2000133549F48C89863509F0BDC16B8D7C8DE9
:101A30008AEA95E0E3CF133429F46B8D7C8D80EB3B
:101A400095E00DC0153529F46B8D7C8D86EB95E006
:101A500006C0103539F46B8D7C8D8FEB95E00E94BC
:101A60009C32E7C11F3409F09EC183E192E00E94DD
:101A7000C5188EE092E00E94A41880918B0590E03A
:101A80000E94D21A89E092E00E94A418C090C90571
:101A9000D090CA05E090CB05F090CC05A701960147
:101AA000C701B6010E944E32882319F06FE671E03B
:101AB0001AC046015701E894B7F82FEF3FEF4FE700
:101AC0005FE7C501B4010E944E32811111C02FEFB2
:101AD0003FEF4FE75FE7C501B4010E94772F18166B
:101AE0003CF463E771E08DEE94E00E9446187DC0FF
:101AF0002FEF3FEF4FE75FE4C701B6010E94493285
:101B000018161CF467E771E0EECF2FEF3FEF4FE7B9
:101B10005FECC701B6010E94772F87FDF3CF20E06D
:101B200030E0A901C701B6010E94772F87FF09C0E5
:101B30006DE28DEE94E00E943F18F7FAF094F7F80A
:101B4000F0942AE037ED43EA5BE3C701B6010E9457
:101B500035314B015C010E941A326B017C010E94FD
:101B60007C2F9B01AC01C501B4010E9434314B01B3
:101B70005C012AE0B701A6018DEE94E00E945B189B
:101B80006EE28DEE94E00E943F1820E030E040E2EB
:101B900051E4C501B4010E94DD2F4B015C010E949C
:101BA0001A326B01E12CF12C2AE0B701A6018DEE6F
:101BB00094E00E945B18C701B6010E947C2F9B0134
:101BC000AC01C501B4010E94343120E030E040E2B4
:101BD00051E40E94DD2F0E941A32AB0160E070E0F8
:101BE0002AE08DEE94E00E945B186BE771E08DEEC9
:101BF00094E00E94461884E092E00E94A41840916C
:101C0000C80550E060E070E02AE08DEE94E00E94AC
:101C10005B186BE771E08DEE94E00E9446188FEF41
:101C200091E00E94A41800E010E0F801E657FA4F96
:101C3000428150E060E070E020E18DEE94E00E948F
:101C40005B180530110511F06AE301C06AE08DEE02
:101C500094E00E943F180F5F1F4F0630110529F7CF
:101C60008AEF91E00E94A4180FE511E01A8309831E
:101C70008091940590919505A0919605B091970556
:101C80008B839C83AD83BE83CE0101960E94EF18A7
:101C900085EF91E00E94A4181A83098380919A0528
:101CA00090919B05A0919C05B0919D058B839C8391
:101CB000AD83BE83CE0101960E94EF1880EF91E0C4
:101CC0000E94A4181A8309838091A0059091A10510
:101CD000A091A205B091A3058B839C83AD83BE83A5
:101CE000CE0101960E94EF188BEE91E00E94A4189D
:101CF0001A8309838091A6059091A705A091A80554
:101D0000B091A9058B839C83AD83BE83CE010196E0
:101D10000E94EF1886EE91E00E94A4181A830983AE
:101D20008091AC059091AD05A091AE05B091AF0545
:101D30008B839C83AD83BE83CE0101960E94EF18F6
:101D400081EE91E00E94A41880EB95E00E94BA1AFF
:101D50008CED91E00E94A41886EB95E00E94BA1ADF
:101D600087ED91E00E94A4188FEB95E00E94BA1ACB
:101D700083ED91E00E94C5185CC08534A1F486EC27
:101D800091E00E94A4182091FC063091FD062115D7
:101D9000310511F422E037E0CE010196821B930B4E
:101DA0000E94D21A46C06EE771E0C7010E949332CA
:101DB000892BE1F48AE8E82E85E0F82E00E010E0B7
:101DC000F70161917F01C8010E94A3300F5F1F4F8F
:101DD00003341105A9F780E090E00E949B309091B8
:101DE0008A05891326C08FEA91E0C4CF1635B9F46D
:101DF00083E891E00E94CD1A83EC91E00E94A41840
:101E000087E891E00E94CD1A81EC91E00E94A4182D
:101E100083E991E00E94CD1A8EEB91E0ABCF8CE983
:101E200091E00E94BA1A8DEE94E00E94F11080E0D9
:101E300005C08DEE94E00E94F11081E06C960FB623
:101E4000F894DEBF0FBECDBFDF91CF911F910F91F0
:101E5000FF90EF90DF90CF90BF90AF909F908F90CA
:101E600008951F920F920FB60F9211248F929F9296
:101E7000AF92BF92CF92DF92EF92FF922F933F9358
:101E80004F935F936F937F938F939F93AF93BF9382
:101E9000CF93DF93EF93FF93C090D402D090D502FD
:101EA000E090D602F090D702C701B6016F5F7F4F76
:101EB0008F4F9F4F6093D4027093D5028093D602C8
:101EC0009093D702E7EDF1E0C0E0D0E021913191AD
:101ED000C20FD31F22E0EF34F207C1F7D093E30221
:101EE000C093E2022091E0023091E1022C173D07FD
:101EF00020F4D093E102C093E0020E947C2F209155
:101F0000D8023091D9024091DA025091DB020E944E
:101F1000DD2F4B015C01BE0180E090E00E947C2F30
:101F20009B01AC01C501B4010E9435314B015C013C
:101F3000C701B6016E5F7F4F8F4F9F4F0E947C2F6E
:101F40009B01AC01C501B4010E94A1316093D8028C
:101F50007093D9028093DA029093DB020E941332CD
:101F6000672B51F484E00E94621261E0892B09F032
:101F700060E084E00E948B128091D6018F5F809395
:101F8000D6018C3328F081E08093E4021092D601D0
:101F9000E091D601F0E0EE0FFF1FE952FE4F1182F3
:101FA0001082FF91EF91DF91CF91BF91AF919F91FF
:101FB0008F917F916F915F914F913F912F91FF9002
:101FC000EF90DF90CF90BF90AF909F908F900F9049
:101FD0000FBE0F901F9018950F931F93CF93DF9311
:101FE0008C01C62F660FDD0B60EB75E0CE010E9401
:101FF0009C3265EA71E0CE010E948832B801CE01C0
:102000000E948832CE01DF91CF911F910F910895E8
:10201000EF92FF920F931F93CF93DF93CDB7DEB76D
:102020002B970FB6F894DEBF0FBECDBF8C017B019E
:10203000FB01E40FF51F10820E94CD1A8DEA91E09A
:102040000E94A418C7010E94BA1A6C2F6F5F89E61C
:1020500091E00E94EC0FBC01C8010E949332892BD1
:1020600021F489E691E00E94510C2B960FB6F8946A
:10207000DEBF0FBECDBFDF91CF911F910F91FF90BB
:10208000EF900895FC01538D448D252F30E0842F6F
:1020900090E0821B930B541710F0CF960895019790
:1020A0000895FC01918D828D981761F0828DDF017A
:1020B000A80FB11D5D968C91928D9F5F9F73928F3B
:1020C00090E008958FEF9FEF0895FC01918D828D30
:1020D000981731F0828DE80FF11D858D90E00895FD
:1020E0008FEF9FEF0895FC01918D228D892F90E055
:1020F000805C9F4F821B91098F73992708958DEE05
:1021000094E00E94731021E0892B09F420E0822FD3
:102110000895FC01848DDF01A80FB11DA35ABF4FA4
:102120002C91848D90E001968F739927848FA689D6
:10213000B7892C93A089B1898C9180648C93938DFD
:10214000848D981306C00288F389E02D80818F7DED
:1021500080830895EF92FF920F931F93CF93DF93A5
:10216000EC0181E0888F9B8D8C8D981305C0E889E8
:10217000F989808185FD24C0F62E0B8D10E00F5F5C
:102180001F4F0F731127E02E8C8DE8120CC00FB675
:1021900007FCFACFE889F989808185FFF5CFCE0168
:1021A0000E948910F1CF8B8DFE01E80FF11DE35ADB
:1021B000FF4FF0820B8FEA89FB898081806207C024
:1021C000EE89FF896083E889F98980818064808352
:1021D00081E090E0DF91CF911F910F91FF90EF9000
:1021E0000895CF93DF93EC01888D8823C9F0EA89A5
:1021F000FB89808185FD05C0A889B9898C9186FD00
:102200000FC00FB607FCF5CF808185FFF2CFA889FC
:10221000B9898C9185FFEDCFCE010E948910E7CF5F
:10222000DF91CF91089580E090E0892B29F00E9402
:102230007F1081110C9400000895833081F028F400
:10224000813099F08230A1F008958730A9F088306C
:10225000B9F08430D1F4809180008F7D03C08091EB
:1022600080008F7780938000089584B58F7702C0B7
:1022700084B58F7D84BD08958091B0008F7703C0B1
:102280008091B0008F7D8093B00008953FB7F8949F
:102290008091D0029091D102A091D202B091D3024C
:1022A00026B5A89B05C02F3F19F00196A11DB11DB1
:1022B0003FBFBA2FA92F982F8827820F911DA11DEC
:1022C000B11DBC01CD0142E0660F771F881F991F29
:1022D0004A95D1F708950895FB0141505109460FE1
:1022E000571FE417F50778F4208130E0322F2227BA
:1022F0006181260F311D820F931F8217930708F407
:1023000001963296EECFE417F50751F4208130E0C4
:10231000322F2227820F931F8217930708F401960A
:1023200008958F929F92AF92BF92CF92DF92EF92D9
:10233000FF920F931F93CF93DF937C018B016C016E
:1023400082E0C80ED11C4701E5E08E0E911CC0E072
:10235000D0E0F60141916F0150E060E070E02AE0CA
:10236000C8010E945B185C016EE2C8010E943F1820
:102370008A0D9B1DC80FD91FC814D90451F7F70146
:10238000458150E060E070E02AE0C8010E945B18DF
:102390008C0F9D1FDF91CF911F910F91FF90EF90B8
:1023A000DF90CF90BF90AF909F908F900895DC0109
:1023B00090E020E030E08AE0FB014191BF0144233E
:1023C00009F150ED540F5A3088F4829FF001839F39
:1023D000F00D11249F0120533109240F311D47FDB9
:1023E0003A952F3F310541F338F312C04E3281F454
:1023F000933071F0FD01E90FF11D22839F5F20E012
:1024000030E0DACF933021F415962C9381E00895D3
:1024100080E008951F920F920FB60F9211242F9310
:102420003F934F935F936F937F938F939F93AF935C
:10243000BF93EF93FF938DEE94E00E948910FF917C
:10244000EF91BF91AF919F918F917F916F915F912C
:102450004F913F912F910F900FBE0F901F901895A5
:102460001F920F920FB60F9211242F938F939F9369
:10247000EF93FF93E091FD04F091FE048081E091E1
:102480000305F091040582FD12C09081809106053C
:102490008F5F8F7320910705821751F0E091060539
:1024A000F0E0E351FB4F958F8093060501C08081DA
:1024B000FF91EF919F918F912F910F900FBE0F90F1
:1024C0001F901895CF93DF93282F30E0F901EE5439
:1024D000FB4F8491F901E256FB4FD491F901E65785
:1024E000FB4FC491CC2391F081110E941D11EC2F60
:1024F000F0E0EE0FFF1FE058FB4FA591B491EC9177
:10250000ED2381E090E021F480E002C080E090E0E3
:10251000DF91CF9108951F93CF93DF93282F30E061
:10252000F901EE54FB4F8491F901E256FB4FD4912F
:10253000F901E657FB4FC491CC23C9F0162F811146
:102540000E941D11EC2FF0E0EE0FFF1FEA58FB4F29
:10255000A591B4918FB7F894111105C09C91ED2FFE
:10256000E095E92302C0EC91ED2BEC938FBFDF9156
:10257000CF911F910895CF93DF9390E0FC01E25635
:10258000FB4F2491FC01E657FB4F8491882361F1B6
:1025900090E0880F991FFC01E459FB4FC591D4913D
:1025A000FC01EA58FB4FA591B491611109C09FB796
:1025B000F8948881209582238883EC912E230BC088
:1025C000623061F49FB7F8943881822F809583231D
:1025D0008883EC912E2B2C939FBF06C08FB7F89465
:1025E000E8812E2B28838FBFDF91CF9108958F92A2
:1025F0009F92AF92BF92CF92DF92EF92FF926B01C8
:102600007C010E9446114B015C01C114D104E1041C
:10261000F104F1F00E944611DC01CB0188199909FF
:10262000AA09BB09883E9340A105B10570F321E0DA
:10263000C21AD108E108F10888EE880E83E0981EDE
:10264000A11CB11CC114D104E104F10419F7DDCFC0
:10265000FF90EF90DF90CF90BF90AF909F908F90C2
:1026600008952FB7F8946091CC027091CD028091BB
:10267000CE029091CF022FBF08951F920F920FB6F6
:102680000F9211242F933F938F939F93AF93BF93F8
:102690008091CC029091CD02A091CE02B091CF0258
:1026A0003091CB0223E0230F2D3720F40196A11D9A
:1026B000B11D05C026E8230F0296A11DB11D209370
:1026C000CB028093CC029093CD02A093CE02B09324
:1026D000CF028091D0029091D102A091D202B0910C
:1026E000D3020196A11DB11D8093D0029093D10217
:1026F000A093D202B093D302BF91AF919F918F91DB
:102700003F912F910F900FBE0F901F9018951F9221
:102710000F920FB60F9211242F933F934F935F9315
:102720006F937F938F939F93AF93BF93EF93FF9399
:10273000E0910301F09104010995FF91EF91BF91A0
:10274000AF919F918F917F916F915F914F913F9149
:102750002F910F900FBE0F901F9018951F920F9200
:102760000FB60F9211242F933F934F935F936F9364
:102770007F938F939F93AF93BF93EF93FF93E091DA
:102780000101F09102010995FF91EF91BF91AF9185
:102790009F918F917F916F915F914F913F912F9179
:1027A0000F900FBE0F901F901895ADE0B4E025E09C
:1027B00014969C91149798130DC095E0899FF00191
:1027C0001124E35FFB4F848114968C931382128251
:1027D00014820895992331F0299FD0011124A35F19
:1027E000BB4FE6CF08950F931F93CF93DF938C01D8
:1027F000EB0160E08AE00E948B128AE38EBD0DB48B
:1028000007FEFDCF0C0F1D1FC017D10739F01EBCEE
:102810000DB407FEFDCF8EB58993F6CF61E08AE057
:10282000DF91CF911F910F910C948B120F931F93F7
:10283000CF93DF931F92CDB7DEB7182F062F60E03E
:102840008AE049830E948B12802F8F71812B8EBD6D
:1028500049810DB407FEFDCF4EBD0DB407FEFDCF7F
:1028600061E08AE00F90DF91CF911F910F910C945E
:102870008B121F93CF93DF93182F1076C12FD0E0C8
:102880002091000130E0C217D30789F043E06FE1E7
:1028900080EA0E941614AE0185E0559547958A9509
:1028A000E1F76FE180E80E94161410930001DF91B8
:1028B000CF911F9108951F93CF93DF9300D0CDB791
:1028C000DEB7182F69837A830E9439144981612FFA
:1028D00080E40E94161461E0610F7A81472F80E442
:1028E0000F900F90DF91CF911F910C941614CF93FE
:1028F000C62FBC0182E00E945B1460E08AE00E9467
:102900008B128AE78EBD0DB407FEFDCFCEBD0DB490
:1029100007FEFDCF61E08AE0CF910C948B12BC01E1
:1029200080E00E945B1460E08AE00E948B128AE3E0
:102930008EBD0DB407FEFDCF1EBC0DB407FEFDCF4E
:1029400061E08AE00E948B128EB508951F93CF93A9
:10295000DF931F92CDB7DEB7182F69830E94391419
:102960004981612F80E40F90DF91CF911F910C94EA
:102970001614CF93DF93C82FD62F60E08AE00E9411
:102980008B128D2F8F71C82BCEBD0DB407FEFDCFDE
:102990001EBC0DB407FEFDCFD7FD08C061E08AE084
:1029A0000E948B128EB5DF91CF9108951EBC0DB49D
:1029B00007FEFDCFF3CFCF93DF931F92CDB7DEB7E6
:1029C000682F69830E943914698180E00F90DF913C
:1029D000CF910C94B914CF93DF93EB01682F84ED62
:1029E0000E94A614BE0186ED0E945B14CFE0D0E0E9
:1029F0008AEE0E94DB1480FF08C06AE070E080E08D
:102A000090E00E94F712219799F7DF91CF910895F6
:102A1000CF92DF92EF92FF920F931F93CF93DF93AA
:102A20006C018B014130510579F4CB010E948F1468
:102A3000682FC601DF91CF911F910F91FF90EF900A
:102A4000DF90CF900C947714EA01C60FD71F7E0158
:102A500081E0E81AF10880E10E945B14B60184E18C
:102A60000E945B140115184048F4E11488E0F80650
:102A700028F07E0181E0E81A88E0F80AB70182E1D7
:102A80000E945B1440E16FE180EA0E94161440E26C
:102A90006FE180E80E9416146FE180E00E94B91493
:102AA00085FF07C061E070E080E090E00E94F712CF
:102AB000F3CFDF91CF911F910F91FF90EF90DF90B7
:102AC000CF900895CF92DF92EF92FF920F931F93D2
:102AD000CF93DF938C0160910D0470910E046150CF
:102AE000784EC12C98E1D92EEDE0F4E080E0C0E012
:102AF000D0E045E09481992349F0499F9001112449
:102B0000235F3B4FD9012D913C9101C09B01E08097
:102B1000F1802E193F090280F381E02D2E1B3F0B1F
:102B20002017310739F4B5E08B9FE0011124C35F12
:102B3000DB4F49C00217130748F42C153D0530F44C
:102B4000489FE0011124C35FDB4F6901911107C069
:102B50002097C9F5CDE0D4E085E0D82E1EC0499F6E
:102B6000F0011124E35FFB4F892FC4CFEA80FB8083
:102B700028813981E20EF31ED89EE0011124C35F43
:102B8000DB4F68817981E616F70639F04A815B816F
:102B9000C7010E940815F982E8828C818111E6CF75
:102BA00020910D0430910E0488819981281B390BE6
:102BB0008A819B81281B390B2150384E2017310701
:102BC00010F480E01AC091E0E2E1F4E02281338168
:102BD000232B29F035969F5F9932C1F7F2CF4A81B6
:102BE0005B8128813981240F351F31832083138332
:102BF00002838C8184839C83892FDF91CF911F91E5
:102C00000F91FF90EF90DF90CF9008950F931F9357
:102C1000DB01E42FA80190E0EF3FF9F065E0E69FCB
:102C2000F0011124E35FFB4F02C0EDEDF4E00190F1
:102C3000F081E02D2E0F3F1F65E0689FF001699F36
:102C4000F00D1124E35FFB4F80819181B9018A0F60
:102C50009B1F1F910F910C940815E091DD04F091DA
:102C6000DE04E20FF31FE11568E0F607F0F29F01C2
:102C70002F5F3740E1CFCF92DF92EF92FF920F9319
:102C80001F93CF93DF937B018A01690125E0829F27
:102C9000C0011124EC01C35FDB4F688179816E0DA7
:102CA0007F1D82E00E945B140A80DB81C02DCE195B
:102CB000DF09CC16DD0608F4E60160E08AE00E9438
:102CC0008B128AE78EBD0DB407FEFDCFC8018C0FB5
:102CD0009D1F0817190741F0F80121918F012EBDA2
:102CE0000DB407FEFDCFF5CF61E08AE00E948B12A4
:102CF000CE01DF91CF911F910F91FF90EF90DF9068
:102D0000CF900895EF92FF920F931F93CF93DF938D
:102D10008B017A018F3FD1F025E0829FE0011124E1
:102D2000C35FDB4F02C0CDEDD4E088819981B8014B
:102D3000680F791F80E00E945B148A819B81801B51
:102D4000910BE816F90690F4C70110C08091DD04DC
:102D50009091DE04860F971F811528E0920718F3E3
:102D6000BC016F5F7740CDEDD4E0E4CFDF91CF9130
:102D70001F910F91FF90EF9008958823A1F09091FB
:102D8000DA04992381F08F3F29F48091DF04909138
:102D9000E004089595E0899FF0011124E35FFB4F63
:102DA00082819381089580E090E00895EF92FF92F0
:102DB0000F931F93CF93DF938091770290E0982F2A
:102DC000882720917802820F911D7C0124E1E21A6C
:102DD000F10848E050E061E872E00E970E946C1143
:102DE000C0919502C695C695CC73D0E0AE0169E856
:102DF00072E00E946C118C01CE15DF0508F04CC00A
:102E0000A7014C1B5D0BBE016E5D7F4F809166027A
:102E10000E948216EC01219760E08AE00E948B12EA
:102E20008AE38EBD0DB407FEFDCFA80160E070E01F
:102E30006C177D07C8F41EBC0DB407FEFDCF2EB580
:102E400030E0322F22271EBC0DB407FEFDCF8EB519
:102E5000280F311D420F531F4217530710F44F5FC5
:102E60005F4F6E5F7F4FE4CF8A016C177D0781F45F
:102E70001EBC0DB407FEFDCF8EB590E0982F8827BD
:102E80008A01080F191F0817190710F40F5F1F4F49
:102E900061E08AE00E948B120115110519F0902F54
:102EA000812F02C08FEF9FEFDF91CF911F910F9184
:102EB000FF90EF90089544E150E065E772E080E014
:102EC00090E00E946C11009721F09827892798279D
:102ED00008958FEF9FEF0895CF92DF92EF92FF92C8
:102EE0000F931F93CF93DF93C09165028C2F827055
:102EF000C1FF0FC02091640230E047E652E060E07D
:102F000070E0809166020E943B16CD7FC0936502FF
:102F100015C0C0916202D0916302209719F0CE01D2
:102F20000E94621580936602882309F471C09E0195
:102F300047E652E060E070E00E943B16F0906602C7
:102F40008091DA04882309F45AC085E0F89EF001E4
:102F50001124E35FFB4FC081D1812197028113814E
:102F60000C0F1D1FCE010E948F14E82E882321F024
:102F700060E0CE010E947714BE0184E00E945B14E1
:102F8000B80186E00E945B148AE0C82ED12C40E88C
:102F90006FE180E80E94161440E86FE180EA0E9429
:102FA00016144AE06CE180EA0E94161448E06FE1D2
:102FB00080E80E94161404E610E08CE10E94DB1405
:102FC0008A7061F40115110559F0015011096AE088
:102FD00070E080E090E00E94F712EFCF012B49F4FF
:102FE00048E06FE180EA0E94161481E0C81AD10817
:102FF00071F6EE2021F06E2DCE010E947714FF2095
:1030000019F08F2D0E94D5131092660281E001C045
:1030100080E0DF91CF911F910F91FF90EF90DF90B3
:10302000CF900895CF92DF92EF92FF920F931F936C
:10303000CF93DF936C017A018B01C0E0D0E0CE1515
:10304000DF0589F0D8016D918D01D601ED91FC91DC
:103050000190F081E02DC6010995892B11F47E01C4
:1030600002C02196ECCFC701DF91CF911F910F9144
:10307000FF90EF90DF90CF9008950E945932DC01CD
:10308000ED91FC910190F081E02D0994611571059D
:1030900079F0FB0101900020E9F73197AF01461B61
:1030A000570BDC01ED91FC910280F381E02D099436
:1030B00080E090E008954F925F926F927F92EF923E
:1030C000FF920F931F93CF93DF93CDB7DEB7A197F6
:1030D0000FB6F894DEBF0FBECDBF7C01FA01CB0165
:1030E00019A2223008F42AE08E010F5D1F4F422EF4
:1030F000512C612C712CBF01A30192010E94C1309F
:10310000F901CA01015011096A3014F4605D01C06F
:10311000695CD8016C93232B242B252B61F7B80114
:10312000C7010E944618A1960FB6F894DEBF0FBEE5
:10313000CDBFDF91CF911F910F91FF90EF907F90C6
:103140006F905F904F9008950F931F93CF93DF93ED
:103150008C01C0E0D0E0F801EC0FFD1F6491662304
:1031600071F0E091ED04F091EE040190F081E02D1A
:103170008DEE94E00995892B11F02196ECCFCE01CC
:10318000DF91CF911F910F910895CF93DF930E940C
:10319000A418EC016BE771E08DEE94E00E944618F4
:1031A0008C0F9D1FDF91CF910895FC018281938147
:1031B000A481B5818093620690936306A093640610
:1031C000B09365068BE597E0909369068093680657
:1031D00010926706109266068DEC95E00895CF93E5
:1031E000DF936DEE74E00E949111EC016BE771E0EA
:1031F0008DEE94E00E9446188C0F9D1FDF91CF91B9
:1032000008958F929F92AF92BF92CF92DF92EF92EA
:10321000FF920F931F93CF93DF9300D000D000D085
:10322000CDB7DEB78C016B017A0159010E943113D1
:10323000DC01CB0186509F4FAF4FBF4F8093E80416
:103240009093E904A093EA04B093EB041092DE0497
:103250001092DD041092E0041092DF048DECEDE09A
:10326000F4E0DF011D928A95E9F781E098E0909300
:103270000E0480930D0461E08AE00E94BB1261E0BD
:103280008AE00E948B1261E08BE00E94BB1261E039
:103290008DE00E94BB1260E08CE00E94BB1261E0F6
:1032A0008AE00E94BB1261E08AE00E948B1260E01B
:1032B0008BE00E948B1260E08DE00E948B1280E513
:1032C0008CBD8DB581608DBD4FEF60E08FEF0E94AA
:1032D000161462E070E080E090E00E94F71262E372
:1032E00070E080E090E00E94F7121092DC041092EF
:1032F000DB0420E1822E912C6DE180E00E94B91464
:1033000081110BC0B1E08B1A910839F06AE070E0CE
:1033100080E090E00E94F712EFCF60E070E088E07C
:103320000E945B1460E070E08CE00E945B146FEF21
:1033300077E08AE00E945B1461EB88E30E94A614A8
:103340006FE370E388E20E945B1469EF77EF80E33C
:103350000E945B146DE070E080EC0E945B1442E31D
:1033600062EC80E80E94161462E17CE086EC0E9428
:103370005B1462E184EC0E94A6146CED75E08AECAB
:103380000E945B1460918C0584EE0E94A6146091EB
:103390008D0585EE0E94A61460918E0582EE0E9436
:1033A000A61460918F0583EE0E94A614609190058B
:1033B00080EE0E94A6146091910581EE0E94A614F1
:1033C00060E071E080E10E94EB148FE10E9439140B
:1033D00040EC6BE180E80E94161444E06FE180E865
:1033E0000E94161466E774E084E10E94EB1482E701
:1033F0000E94DB148F3F09F0BAC01092DA0480916A
:103400008C058093E20480918D058093E304809184
:103410008E058093E40480918F058093E50480916C
:1034200090058093E604809191058093E70480E005
:10343000E82FF0E0EE0FFF1FEC5FFB4F11821082D0
:103440008F5F8430A9F780E09EE1989FF0011124FE
:10345000E457FC4F118E8F5F8430B9F780930C04D2
:1034600080E094E090938B0380938A031092890309
:103470009BE080918903883068F4989FF0011124C3
:10348000EF5CFC4F10821182128213828F5F809357
:103490008903EFCFF50192805381B4819581F701C3
:1034A000A2818381B4804581F601C280D380E4800B
:1034B000F580F801248130E0322F22276581262B08
:1034C000322723273227628170E0762F6627138107
:1034D000612B76276727762770932E0360932D0341
:1034E0003093300320932F03282F30E03A2B3827D6
:1034F0002327322730932A0320932903242F30E0F7
:103500003B2934272327322730932C0320932B0386
:10351000252F30E0392935272327322730932603FA
:1035200020932503892F90E09B2B982789279827A4
:103530009093280380932703C0929006D09291061F
:10354000E0929206F092930626960FB6F894DEBFAC
:103550000FBECDBFDF91CF911F910F91FF90EF90E4
:10356000DF90CF90BF90AF909F908F900895809301
:10357000DA0445CFCF93DF93BC018DEE94E00E9437
:103580004618EC016BE771E08DEE94E00E9446185E
:103590008C0F9D1FDF91CF910895BC018DEE94E0BB
:1035A0000C944618CF92DF92EF92FF92CF93DF9365
:1035B0006C01990FEE08FF08F7FE16C06DE28DEE64
:1035C00094E00E943F18EC0144275527BA014C199A
:1035D0005D096E097F092AE08DEE94E00E945B1878
:1035E0007C01EC0EFD1E08C02AE0B701A6018DEE9D
:1035F00094E00E945B187C016BE771E08DEE94E033
:103600000E9446188E0D9F1DDF91CF91FF90EF9085
:10361000DF90CF900895CF93DF93DC014E5F5F4F33
:10362000FC019F012A1B3B0B9191992339F0EB017F
:10363000C40FD51F98834F5F5F4FF3CFCA01821B22
:10364000930B680F791FFB013297308331962083EB
:10365000CA01DF91CF910895CF92DF92EF92FF924E
:103660000F931F93CF93DF9300D000D0CDB7DEB779
:10367000FA0130E09E2F9F77EE0FEF2FEE1FFF0B2A
:10368000F195309709F0906821E0230FA1E0B0E0B8
:10369000AC0FBD1FA30FB11D9C93309711F0322FBB
:1036A000E9CF30E0DB01A21BB30B14968C93CE0163
:1036B00001966C0180E090E08217930764F4F601B4
:1036C00011916F017C01E21AF30AE60EF71EF70171
:1036D00015830196F1CF8091D1059091D2052F5F8E
:1036E0003F4F8901040F151FFC0120813181F90131
:1036F00022813381A801BD01F90109957C010E9455
:103700003113609355067093560680935706909335
:10371000580681E0E016F10609F080E00F900F9066
:103720000F900F90DF91CF911F910F91FF90EF902D
:10373000DF90CF9008958091D1059091D2050097A8
:1037400059F1DC01ED91FC910688F789E02D09958E
:10375000811124C080916C0690916D06892BE1F453
:103760008DEF9FEF90936D0680936C068091D1054D
:103770009091D205DC01ED91FC910680F781E02D5E
:1037800009958091D1059091D205DC01ED91FC91D4
:103790000488F589E02D099580E0089581E0089579
:1037A000CF93DF931F92CDB7DEB7DC01ED91FC9193
:1037B0000288F389E02D41E050E0BE016F5F7F4F4A
:1037C0000995181619061CF4898190E002C08FEF44
:1037D0009FEF0F90DF91CF910895EF92FF920F939B
:1037E0001F93CF93DF93EC01E881F981008CF18D79
:1037F000E02D09958823B9F08C859D857C012FEFFC
:10380000E21AF20A8C010A5F1F4FC0E0D0E0F70114
:1038100081917F010E94BD16C80FD91FE016F106E5
:10382000B1F7CE0102C080E090E0DF91CF911F910F
:103830000F91FF90EF9008950F931F93CF93DF9315
:103840001F92CDB7DEB78C01DC01ED91FC91008CAD
:10385000F18DE02D09958823B1F0D8011C96ED91EA
:10386000FC911D978181882371F041E050E060E078
:1038700070E00E948216BE016F5F7F4F0E94F313BB
:10388000898190E002C08FEF9FEF0F90DF91CF9181
:103890001F910F910895CF93DF93EC0188818111DF
:1038A0000E94D513DE011196FE01CE0104962D91E2
:1038B0002193E817F907D9F71C82DF91CF9108957A
:1038C0004F925F927F928F929F92AF92BF92CF92D0
:1038D000DF92EF92FF920F931F93CF93DF937C01C0
:1038E0004B01EA01DC01ED91FC91008CF18DE02DA2
:1038F0000995882309F475C0D7011C96ED91FC91B8
:103900001D978181882309F46FC06E018EE1782EA6
:103910008E010C191D09080D191DD7011C96ED917A
:10392000FC911D97A60160E070E081810E948216E3
:103930005C01B8010E94F313F70144845584D2015D
:1039400011961C91812F0E94BD16A816B90681F50B
:10395000CA18DB08C20101960E944B1CF701A4851E
:10396000B5858C91282F30E02F70729EF001739EE8
:10397000F00D1124E457FC4F918D94FF05C0982F52
:10398000907611F480688C93D7011C96ED91FC9190
:103990001D97818181111FC0808186FF05C0108223
:1039A0001D961C921E921C97CE018C199D091EC05B
:1039B000B5E01B9FF0011124E35FFB4F80819181F3
:1039C0008A0D9B1D91838083828193818A199B0933
:1039D0009383828304C0C114D10409F099CFCE012E
:1039E00005C08FEF9FEF02C080E090E0DF91CF91A4
:1039F0001F910F91FF90EF90DF90CF90BF90AF900D
:103A00009F908F907F905F904F900895CF92DF921C
:103A1000EF92FF920F931F93CF938091DA04882344
:103A200009F423C21091F906111166C089E30E94BE
:103A3000DB149091DA04992309F45CC0882309F41B
:103A400059C06091DB047091DC047B0126E0E20E3A
:103A5000F11CE11438E0F30628F07B0149EFE41A89
:103A600047E0F40A80E00E945B1460E08AE30E9471
:103A7000B91490E09093DC048093DB0460E08AE367
:103A80000E94B9142091DB043091DC04382B309370
:103A9000DC042093DB0460E08AE30E94B914C82FA1
:103AA00060E08AE30E94B914082F60E08AE30E9474
:103AB000B914D82E40E46EE180E80E94161460919B
:103AC000DB047091DC04D7FE12C0611558E0750765
:103AD00070F4F092DE04E092DD048C2F90E0902BE5
:103AE00004979093E0048093DF041FEF03C08CE001
:103AF0000E945B141093F906C091F906CC2309F4D7
:103B00004FC181E0809365028C2F0E94BD16909377
:103B1000630280936202892B09F435C142E650E0CA
:103B200060E070E08C2F0E94821667E672E00E94CF
:103B3000F31300917302109174020830110509F01B
:103B40006EC0C093660280916202909163020E97EC
:103B500090936302809362022091810230918202ED
:103B6000E0912D03F0912E03AF014227532780915E
:103B700025039091260384239523892B09F042C0C5
:103B8000409183025091840260912F037091300321
:103B9000DB01A427B52780912703909128038A236E
:103BA0009B23892B79F580918502909186028E174F
:103BB0009F0771F48091870290918802861797077A
:103BC00039F46DE672E081E892E00E9469041AC05F
:103BD00080E09BE08830A1F0989FF0011124EF5C19
:103BE000FC4F608171812617370741F46281738130
:103BF0004617570719F480938903E3CF8F5FEACF05
:103C00008093890381E00E94060680916202909170
:103C10006302892B09F4B7C00E94D204B2C00830F5
:103C200086E0180709F0AFC08091620290916302AC
:103C300010926302109262028A9708F49CC08091ED
:103C40007B0290917C028115A1E09A0729F08115F1
:103C5000924009F474C08FC020918D0230918E0281
:103C600080912D0390912E032817390709F083C006
:103C700020918F023091900280912F039091300318
:103C80002817390709F077C06DE772E083E892E002
:103C90000E94690480E092E090937C0280937B0212
:103CA00086E0EDE7F2E0A7E8B2E001900D928A9598
:103CB000E1F786E0E2EEF4E0ADE7B2E001900D92CC
:103CC0008A95E1F786E0E2EEF4E0ADE6B2E001903D
:103CD0000D928A95E1F786E0E7E8F2E0A7E6B2E028
:103CE00001900D928A95E1F7809183029091840270
:103CF00090938E0280938D0280918502909186022E
:103D00009093900280938F0280912D0390912E03C7
:103D1000909384028093830280912F0390913003CB
:103D2000909386028093850210937402009373022D
:103D30008AE290E090936302809362021CC020911B
:103D40008D0230918E0280912D0390912E032817C1
:103D5000390789F420918F023091900280912F03CE
:103D6000909130032817390731F46DE772E083E84A
:103D700092E00E9469048091620290916302892B13
:103D800011F00E946C178091650280FF09C060915C
:103D9000DB047091DC048CE00E945B141092F90645
:103DA0000E9431136B017C018091E8049091E90439
:103DB000A091EA04B091EB04A7019601281B390BEE
:103DC0004A0B5B0BDA01C90180959095A095B095DF
:103DD0008827B7FD83959927AA27BB27C82F0CE80A
:103DE00013E01093B4060093B306CC2311F082E0E5
:103DF00017C00115110519F1D8015C96ED91FC91E0
:103E00005D973097D1F085859685A785B089A70104
:103E10009601281B390B4A0B5B0B57FD10C083E042
:103E20000E9406068091620290916302892B39F00C
:103E30000E94D2040E946C1702C0F801E4CF025E17
:103E40001F4F34E00430130761F6CC2371F0D70123
:103E5000C60186509F4FAF4FBF4F8093E8049093A9
:103E6000E904A093EA04B093EB04CF911F910F9162
:103E7000FF90EF90DF90CF9008950F931F93CF9313
:103E8000DF93EC018C010B5F1F4F888181110E9431
:103E9000D5131992C017D107C1F7DF91CF911F91A8
:103EA0000F910895CF93DF93EC01E881F981008CA5
:103EB000F18DE02D0995882339F08C859D8501963B
:103EC000DF91CF910C943D1FDF91CF910895CF9258
:103ED000DF92EF92FF920F931F93CF93DF93E090C7
:103EE000B306F090B406D7015C96CD91DC915D9756
:103EF000D090B2062097B9F5D6FE6AC0E5EBF6E0A1
:103F000080E090E02081211128C041E1489F90018C
:103F1000499F300D1124E901CB54D94FA7014C58CA
:103F20005340559547956FEE7EEE469FC001479FE3
:103F3000900D569F900D112480618883F901EA54F9
:103F4000F94F80E1DF011D928A95E9F7209709F486
:103F50003FC0F701D58FC48F06C00196719684309B
:103F6000910581F635C0D1FE07C080916202909123
:103F70006302892B09F050C0888187FF0DC08F77BD
:103F800088838D2D82608093B206D70159968C91DB
:103F900059978F7E59968C931091B206B12FB071BC
:103FA000DB2E14FF7EC0CE0106960E943D1F898144
:103FB000882309F479C0F701848195819F838E83DA
:103FC000888180648883D7015D961C921E925C97DD
:103FD000E12CF12C6091B0067091B106F092AF0621
:103FE000E092AE061E141F0454F48091AC0690912A
:103FF000AD066817790719F0A7010E946632F092A2
:104000006302E0926202DF91CF911F910F91FF90C6
:10401000EF90DF90CF9008958881807609F0ACCF43
:104020008E010F5F1F4FC12CD8018C91811129C0C7
:1040300020916202309163022115310519F0C90106
:104040000E946215F80180838823D9F000916202F2
:10405000109163022091B0063091B106275632408C
:104060004091F90660E070E00E940616F4E0CF127D
:1040700083CFD70159968C915997806159968C932B
:104080007BCFC3940F5F1F4FB5E0CB12CDCF809194
:1040900065028E7F80936502F701818D8061818F3B
:1040A0006BCF17FF03C07FCF18828DCF10FF04C0E6
:1040B000CE0106960E944B1C1C7009F443C0EE8191
:1040C000EE2309F43FC08F8181110FC0EB84FC8483
:1040D000E114F10409F47ECFB5E0EB9FF001112467
:1040E000E35FFB4FF382E28207C08E2F0E94BD1672
:1040F0007C01892B09F46ECF8091B0069091B106B6
:104100008756924080936402F701E80FF11DCF01BA
:10411000EF2B19F00E946215D82ED0926602DD2096
:1041200009F458CF6091640270E0870120E030E02C
:104130004E818D2D0E9406168091650282608093CB
:10414000650248CF888185FF43CF8E8181110AC0E7
:104150001882D7015D961C921E925C9780E1809335
:10416000B20636CFF701818D8061818F31CF8F927A
:104170009F92AF92BF92CF92DF92EF92FF920F93F6
:104180001F93CF938C015B017A016A014C0187E098
:10419000880E911C0E94061D0115110509F452C0DC
:1041A000F8018081807609F04DC0F401C1E0819171
:1041B000811102C0C15004C0CF5FC530C1F7C4E057
:1041C000F801EC0FF11D868181110DC080E092E0B5
:1041D0000E946215F801EC0FF11D86838823D1F24D
:1041E000F80114861386A7014C195D094A0D5B1D61
:1041F000F801638574859601EC0FF11D86810E949C
:104200003B16C81AD90AF80123853485820F931FFB
:10421000948783871C141D042CF4C43009F4BACF8E
:10422000CF5FD4CF0E943113DC01CB010A96A11DD0
:10423000B11DF80185879687A787B08BC7018C19B8
:104240009D0902C080E090E0CF911F910F91FF90F7
:10425000EF90DF90CF90BF90AF909F908F90089598
:10426000CF92DF92EF92FF92CF93DF93EC010E9407
:1042700031136B017C018091D1059091D205DC0155
:10428000ED91FC910084F185E02D0995892B79F45D
:104290000E943113AB01BC014C195D096E097F0905
:1042A00048395A436105710530F380E00DC08091B3
:1042B000D1059091D205DC01ED91FC910284F3854A
:1042C000E02D0995888381E0DF91CF91FF90EF90F9
:1042D000DF90CF900895EF92FF920F931F93CF93AB
:1042E000DF937C018B01EB0109900020E9F7219716
:1042F000C61BD70B0E949B1B8823B1F1F7010190CD
:104300000020E9F73197EE19FF09CE010796E80F73
:10431000F91FE138F10540F545E050E063ED75E047
:10432000C7010E940B1BF80120E030E02C173D076D
:1043300059F04191D901A80FB91FA353BA4F16964E
:104340004C932F5F3F4FF2CF25503109A901480F01
:10435000591F63ED75E080E3DF91CF911F910F91BD
:10436000FF90EF900C942C1B80E0DF91CF911F9178
:104370000F91FF90EF9008955F926F927F928F92CE
:104380009F92AF92BF92CF92DF92EF92FF920F93E4
:104390001F93CF93DF931F92CDB7DEB74C0183ED10
:1043A00095E00E943021882309F441C07090D30524
:1043B000198201E010E0A12CB12CC12CD12C760186
:1043C000C394CE0101960E943021882381F10F5FB2
:1043D0001F4F8981F801E353FA4F8583282F2F77E8
:1043E00030E02C9DA0012D9D500D3C9D500D1124C1
:1043F000A40EB51E37E0CC0CDD1CEE1CFF1C3A955C
:10440000D1F787FF17C005301105D9F68FEF9FEF61
:1044100090936D0680936C068091D1059091D205A2
:10442000DC01ED91FC910488F589E02D099580E08F
:1044300090E07CC0872D807F55245394803309F011
:10444000512C8FEF800FF4018083552021F1C8019A
:104450008D529A4F0E943021882349F3C8018C5213
:104460009A4F0E943021882311F30E5F1F4FD40111
:10447000EC91F0E0E353FA4FE780F12CFE2CEE24B0
:104480008085E80EF11C8091D30581FF08C0B2E061
:10449000EB0EF11C04C080E0E12CF12C01C082E0A5
:1044A000C82ED12CC01AD10A9EEF692E77247A9497
:1044B000C601800F911F8A159B0568F5CE010196F4
:1044C0000E943021882309F4B2CF80916A0690912E
:1044D0006B060097A9F0552099F0F4012081A30103
:1044E000421B51099A01200F311FE216F30640F4D6
:1044F000DC01ED91FC910190F081E02D698109953D
:104500000038110528F48981F801E353FA4F8683B6
:104510000F5F1F4FCDCF80916A0690916B06892B5C
:1045200021F40138110508F082CFC8010F90DF9106
:10453000CF911F910F91FF90EF90DF90CF90BF90A0
:10454000AF909F908F907F906F905F900895FC0147
:104550002381260F20935402A72FBB2792819A0F05
:104560009093530231813093520240814093510223
:10457000E92FF0E0EA17FB0748F481E0830F80930E
:104580005202811103C04F5F4093510230E0772700
:104590002617370788F49F5F9093530291110CC040
:1045A000809152028F5F80935202811105C08091E9
:1045B00051028F5F8093510208952091B30630918C
:1045C000B406BC01C90108960E94A722E091B30677
:1045D000F091B406A1E5B2E08C91808711968C91A0
:1045E0001197818712968C911297828713968C91DE
:1045F00083870895CF93DF93CDB7DEB7AF970FB61C
:10460000F894DEBF0FBECDBF789484B5826084BDC0
:1046100084B5816084BD85B5826085BD85B58160C6
:1046200085BD80916E00816080936E001092810044
:1046300080918100826080938100809181008160FF
:1046400080938100809180008160809380008091C0
:10465000B10084608093B1008091B000816080934C
:10466000B00080917A00846080937A0080917A0013
:10467000826080937A0080917A00816080937A00D2
:1046800080917A00806880937A001092C100E09156
:10469000FD04F091FE0482E08083E091F904F09142
:1046A000FA041082E091FB04F091FC0480E1808325
:1046B00010920505E0910105F091020586E08083E6
:1046C000E091FF04F0910005808180618083E0919A
:1046D000FF04F0910005808188608083E091FF04F1
:1046E000F0910005808180688083E091FF04F09163
:1046F000000580818F7D808382E095E00E94A41870
:1047000083E891E00E94CD1A8CEE94E00E94C518D7
:1047100060E083E00E94BB1262E085E00E94BB1271
:1047200060E08EE00E94BB1261E084E00E94BB1258
:1047300083E08093050161E084E00E948B1280E0B9
:1047400090E00E949B3090918A058917D9F10E94D0
:10475000270CF8941092800010928100109285002E
:104760001092840088E09DE39093890080938800F4
:1047700080918100886080938100809181008560B4
:104780008093810080916F00826080936F008DEF35
:1047900092E09093040180930301809169008C6002
:1047A00080936900E99A789485E00E94621221E082
:1047B000892B09F420E020930601211115C082ED18
:1047C00094E014C02AE8E22E25E0F22E00E010E08A
:1047D000C8010E949B30D7018D937D010F5F1F4F51
:1047E00003341105A9F7B3CF8FED94E00E94C518EB
:1047F00080910601882309F489C080918B05882364
:1048000051F099E288E10FB6F894A8958093600082
:104810000FBE9093600086EC94E00E94A4180FE510
:1048200011E01A8309838091A6059091A705A091B4
:10483000A805B091A9058B839C83AD83BE831A8B99
:10484000098B8091A0059091A105A091A205B0913E
:10485000A3058B8B9C8BAD8BBE8B1AA309A3809178
:104860009A0590919B05A0919C05B0919D058BA305
:104870009CA3ADA3BEA318A70FA38091940590910C
:104880009505A0919605B091970589A79AA7ABA722
:10489000BCA79E012F5F3F4FAE014F5E5F4FBE0131
:1048A0006F5D7F4FCE0187960E94011930912D03D5
:1048B00020912E0390912F03809130031A83098356
:1048C0003B832C839D838E83CE0101960E94EF183B
:1048D0008EE696E09093D2058093D10588E090E132
:1048E00090935F0680935E061A8309838091AC05DE
:1048F0009091AD05A091AE05B091AF058B839C83DF
:10490000AD83BE83CE0101960E94D518FE0131967B
:104910001F019E01285F3F4F3EA72DA78DEE94E01B
:104920000E947310892B69F18DEE94E00E94511062
:104930008A3089F08D30B9F0209122033091230321
:10494000F901EA51FD4F80832F5F3F4F30932303DE
:104950002093220308C086EE92E00E94510C109230
:10496000230310922203E0912203F0912303EA51E2
:10497000FD4F10826AE070E080E090E00E94F71244
:10498000CDCF8091E502882381F061E084E00E9430
:104990008B1264E670E080E090E00E94F71260E025
:1049A00084E00E948B121092E502109106011123FF
:1049B00009F4E3C10E94061D80912403882331F08D
:1049C00085E00E946212019709F4DFC18091E40240
:1049D00081110AC0809124038111ADC085E00E943D
:1049E0006212892B09F0A7C00E949B1B811149C24A
:1049F00060916606709167068091D1059091D2050D
:104A00004091680650916906DC01ED91FC916115B9
:104A1000710509F4BDC10088F189E02D0995813047
:104A2000910509F027C29093540680935306EDE058
:104A3000F1E0D10187E001900D928A95E1F7F10153
:104A4000A8EDB5E081918D934DA55EA5E417F5071E
:104A5000C9F786EB95E0892B09F4AFC1AFEBB5E060
:104A6000AB2B09F4ACC182EC8093DF051092E0051A
:104A70008FE08093E105E0EBF5E001900020E9F79D
:104A8000CF01805A95408138910508F0E7C14FE089
:104A900050E063ED75E080EB95E00E940B1BE6EBC8
:104AA000F5E0309709F08DC1AC014550510963ED37
:104AB00075E080E10E942C1B0E9431136093550623
:104AC0007093560680935706909358066093590644
:104AD00070935A0680935B0690935C068091D10593
:104AE0009091D205DC01ED91FC910084F185E02DDF
:104AF0000995892B09F490C1CE0141960E94BC21F1
:104B0000049709F0ABC18091D6058111A2C10E9422
:104B100031136093590670935A0680935B06909305
:104B20005C0610925D0610926D0610926C061111D3
:104B3000A8C11092E4020E949B1B882309F41DC1A6
:104B40000E9431132B013C018091590690915A0625
:104B5000A0915B06B0915C06A3019201281B390B62
:104B60004A0B5B0BDA01C90189399A43A105B105EA
:104B7000A8F48091550690915606A0915706B091E1
:104B80005806A3019201281B390B4A0B5B0BDA0173
:104B9000C90189399A43A105B105C8F120915D0683
:104BA0008091D1059091D205222371F04CEF5FEFF7
:104BB00050936D0640936C06DC01ED91FC910488E6
:104BC000F589E02D0995D9C020EC2093D3051092EA
:104BD000D405DC01ED91FC910280F381E02D42E0EF
:104BE00050E063ED75E009954092550650925606E7
:104BF00060925706709258064092590650925A0693
:104C000060925B0670925C0681E080935D06809105
:104C1000D1059091D205DC01ED91FC910084F185E4
:104C2000E02D0995892B09F4A8C0C1010E94BC217F
:104C30004C01892B09F49FC04092590650925A06A4
:104C400060925B0670925C068091D305807F803312
:104C500009F075C080915E0690915F06892B09F47A
:104C60008CC0E980F12CF701E353FA4F078110E083
:104C7000102F00278085080F111DF701EB52FA4F06
:104C80005F01B7016A527A4FA801CF010E946F32CB
:104C900098012E0D3F1DF901E353FA4F10868091C4
:104CA000D30586708FA7A0915E06B0915F06823013
:104CB000B9F5C184D12CDC2CCC248285C80ED11C42
:104CC0004BEF5FEF4E195F09401B510B480D591D0B
:104CD000B90168527A4FC501FD01099580E48093BE
:104CE000D3052FA52093D405D092D505C092D60523
:104CF0008091D1059091D205DC01ED91FC9102806B
:104D0000F381E02D44E050E063ED75E009954092B9
:104D100055065092560660925706709258062DC05E
:104D20004DEF5FEF4E195F09401B510B480D591DA8
:104D3000B9016A527A4FC501FD0109951EC0803C38
:104D4000A9F480ED8093D3051092D4058091D1050C
:104D50009091D205DC01ED91FC910280F381E02D70
:104D600042E050E063ED75E0099507C0803D29F40D
:104D700010925D0602C00E949B1B80918B058823C8
:104D800009F0A8950E941311C9CD109224031ECEDC
:104D90000684F785E02D2FE531E03A832983C09022
:104DA0006206D0906306E0906406F0906506CB82C0
:104DB000DC82ED82FE82B10131CE82E055CE82E806
:104DC00053CE01900020E9F79C012E0F3F1F255B79
:104DD00035402138310508F041C0AC0163ED75E084
:104DE00086EB95E00E940B1BEFEBF5E0309709F4A2
:104DF0005BCE01900020E9F79C012E0F3F1F2E5B38
:104E000035402138310550F5AC0163ED75E08FEB8D
:104E100095E00E940B1B48CE0E943113C0905906AA
:104E2000D0905A06E0905B06F0905C06DC01CB0166
:104E30008C199D09AE09BF0988399A43A105B105AE
:104E400008F44CCE2CEF3FEF30936D0620936C06A8
:104E500005C090E090936D0680936C068091D1051B
:104E60009091D205DC01ED91FC910488F589E02D4B
:104E700009955FCEEEEFFFEFF0936D06E0936C06C1
:104E800058CE80EB95E00E94CD1A88E395E00E9411
:104E9000A4184AE0BE016F5E7F4F8091E2029091BC
:104EA000E3020E942B2B622D87EA91E00E94EC0F17
:104EB000BE016F5E7F4F0E946B2182E395E00E94EE
:104EC000A418CE0141960E94CD1A4AE0BE016F5E41
:104ED0007F4F8091E0029091E1020E942B2B622D86
:104EE0008BEA91E00E94EC0FBE016F5E7F4F0E9443
:104EF0006B218CE295E00E94A418CE0141960E949D
:104F0000CD1A6091DC027091DD028091DE029091F9
:104F1000DF022AE0AE014F5E5F4F0E94362B622D0A
:104F20008FEA91E00E94EC0FBE016F5E7F4F0E94FE
:104F30006B2186E295E00E94A418CE0141960E9462
:104F4000CD1A6091D8027091D9028091DA029091C5
:104F5000DB028E010F5E1F4F22E04AE00E94A22971
:104F6000622D83EB91E00E94EC0FB8010E946B214F
:104F700080E295E00E94A418C8010E94CD1A6091B9
:104F8000D4027091D5028091D6029091D70226E08A
:104F9000A8010E94362B622D87EB91E00E94EC0F56
:104FA000B8010E946B218AE195E00E94A418C80113
:104FB0000E94CD1A80910501F0E48F9FC001112459
:104FC00080937C0080917A00806480937A00809145
:104FD0007A0086FDFCCF609178008091790070E0C6
:104FE000782B072E000C880B990B0E947E2F20E057
:104FF00030E048EC52E40E94DD2F6B017C016091AF
:10500000C80570E080E090E00E947E2F9B01AC011B
:10501000C701B6010E94A1310E941332DC01CB010D
:105020004AE0BE016F5E7F4F0E942B2B622D8BEBFF
:1050300091E00E94EC0FBE016F5E7F4F0E946B21DA
:1050400084E195E00E94A418CE0141960E94CD1AF9
:105050006091C9057091CA058091CB059091CC05EE
:105060008E010F5E1F4F22E046E00E94A229622DB2
:105070008FEB91E00E94EC0FB8010E946B218EE053
:1050800095E00E94A418C8010E94BA1A622D89E610
:1050900091E00E94EC0F8C01FC0101900020E9F7E7
:1050A0009F01281B390B285F3F4F2138310580F5C0
:1050B0000E949B1B882361F18091530690915406B6
:1050C000019629F0909354068093530606C021E080
:1050D00030E030935406209353068091530690910C
:1050E00054069093D8058093D90547E050E063EDCE
:1050F00075E0C8010E940B1BFC01E353FA4F1682B6
:10510000AC014450510963ED75E082E80E942C1B0C
:1051100061E084E00E948B1264E670E080E090E041
:105120000E94F71260E084E00E948B1281E080937D
:105130002403FFCCCF93DF93ECE7F6E08FE591E01B
:10514000918380831282138214821582EDEEF4E043
:105150001382128248EE53E060E070E0448355838E
:10516000668377832FE131E03183208325EC30E0C3
:105170003587248724EC30E03787268720EC30E021
:10518000318B208B21EC30E0338B228B22EC30E012
:10519000358B248B26EC30E0378B268B118E128ECC
:1051A000138E148EE2E8F6E09183808312821382DC
:1051B00014821582E8E8F6E09183808312821382DC
:1051C00014821582E4E9F6E09183808312821382CF
:1051D00014821582EEE8F6E09183808312821382B6
:1051E00014821582EAE9F6E09183808312821382A9
:1051F00014821582E0EAF6E09183808312821382A2
:1052000014821582E6EAF6E091838083128213828B
:1052100014821582EEE6F6E01382128244835583EF
:10522000668377832DE331E03183208315861486EE
:10523000EDECF5E01382128221E331E0318320832B
:105240009093610680936006109262061092630646
:1052500010926406109265062FEF3FEF30936D06B3
:1052600020936C061582148210926B0610926A06C7
:1052700010925F0610925E06CAE8D5E029E92883FD
:10528000198226E0E4E1F1E0ACE8B5E001900D928E
:105290002A95E1F79987888730EC3A8728EA2B87A7
:1052A0001C8642E14D879F878E8744ED488B4BE1FA
:1052B000498B48E24A8B40EF4B8B9D8B8C8B3E8B0E
:1052C0002F8B188E4EEF498F9B8F8A8F4FEF4C8F0D
:1052D0004D8F4E8F1F8E99A388A33AA32BA31CA298
:1052E00084EB8DA3E0EBF5E083E497E4ADE4B0E07C
:1052F00080839183A283B3831582148289E0E3ECD7
:10530000F1E0A6EBB5E001900D928A95E1F789E016
:10531000ECECF1E0AFEBB5E001900D928A95E1F78E
:105320008CE88093C8058DEC9CECA9E1B3E48093F4
:10533000C9059093CA05A093CB05B093CC05DF9126
:10534000CF910895EF920F931F93CF93DF93E801CE
:1053500047FD02C034E001C034E1E42F440FFF0BED
:10536000F7FF03C0F195E195F109E32E022F2E2FEF
:10537000AE010E94892BCE01DF91CF911F910F9139
:10538000EF900895A6E0B0E0E8ECF9E20C94EE307E
:105390005C016B017A016115710519F0DB018D93D8
:1053A0009C93E114F10429F0C7010297839708F058
:1053B000DCC03501BFEF6B1A7B0AF5011081812F2C
:1053C00090E00E94F62A892B11F05301F2CF1D3292
:1053D00049F43501F2E06F0E711CD50111961C9154
:1053E00001E009C01B3231F43501B2E06B0E711CD3
:1053F000F501118100E0E114F10409F4C4C0F0E109
:10540000EF16F10489F4103399F5D3018C918F7D57
:10541000883509F0B2C011961C91B2E06B0E711C78
:10542000026050E1E52EF12CEAE0EE16F10409F4F9
:10543000B0C0F0E1EF16F104D9F028E0E216F10473
:1054400051F438E0E32EF12C88248A94982CA82C6F
:105450004FE1B42E13C06FEF7FEFCB0197010F2CFC
:10546000000C440B550B0E94C13049015A0106C083
:1054700088248A94982CA82C2FE0B22E7E826D82EC
:1054800060E020E030E0A90127010F2C000C660845
:1054900077082D803E80E0EDE10FEA3060F08FEB81
:1054A000810F8A3110F4E9EC05C08FE9810F8A3150
:1054B00090F5E9EAE10F8E2F90E08E159F055CF5DF
:1054C0006F3F09F182169306A406B506D8F0C30112
:1054D000B2010E94B1302E2F30E040E050E029832D
:1054E0003A834B835C83260F371F481F591F8981DE
:1054F0009A81AB81BC81281739074A075B0710F0F6
:1055000061E001C06FEFED81FE813196FE83ED8396
:10551000D1011C91BECFC114D10489F0662339F0AA
:105520008D819E810197F6019183808308C001FFE0
:1055300006C08D819E810297D6018D939C9300FFBA
:1055400007C050954095309521953F4F4F4F5F4F85
:1055500067FF10C082E290E09093010780930007FC
:105560006FEF7FEF8FEF9FEF1BC060E070E080E098
:1055700090E016C0B901CA0113C010E3E114F104B0
:1055800009F45FCF51CF103309F43FCF9AE0E92EF1
:10559000F12C89E9882E982CA82C89E1B82E6ECFA1
:1055A0002696E2E10C940A31662777270C94172D92
:1055B000FC0188279927E89421912032E9F32930CA
:1055C00010F02E30C8F32B3241F02D3239F46894AC
:1055D00004C00E94452B820F911D219120532A3037
:1055E000C0F31EF4909581959F4F089591110C94EE
:1055F0004C2F803219F089508550C8F708954AEF32
:1056000056E00E94042B0895FA01A191B081009701
:1056100019F41097E1F0CD01DC01CD010D900020CF
:1056200011F4C00113C0FB012191222319F02015B0
:10563000D9F7F3CFFB012191201519F41E92119691
:1056400006C02223C1F70D900020A1F7D001FA0176
:10565000A193B0830895BB274A3031F4992322F4F3
:10566000BDE2909581959F4F0C94702BBB272A30FB
:1056700051F4992342F4BDE290958095709561951F
:105680007F4F8F4F9F4F0C944E2B7AE0979F902D1A
:10569000879F802D910D11240895BB27FA01A62F15
:1056A0006217710581059105330B30FB66F0AA275F
:1056B000660F771F881F991FAA1FA21710F0A21B41
:1056C00063953850A9F7A05DAA3308F0A95DA193AE
:1056D00036F7B111B1931082CA010C94672FBB2722
:1056E000FB015527AA27880F991FAA1FA41710F09E
:1056F000A41B83955051B9F7A05DAA3308F0A95DAA
:10570000A193009779F7B111B1931192CB010C9449
:10571000672F4F925F926F927F929F92AF92BF924C
:10572000CF92DF92EF92FF920F931F93CF93DF936D
:10573000CDB7DEB729970FB6F894DEBF0FBECDBF49
:105740006A01122FB02E2BE3201720F0FF24F394D0
:10575000F00E02C0BCE3FB2E0F2D27E0AE014F5F21
:105760005F4F0E94742EAC018981982F99709130FF
:1057700031F0E1FC06C0E0FE06C090E205C09DE20B
:1057800003C09BE201C090E0EE2DE07183FF3CC0BE
:10579000911102C083E001C084E0811718F4212F29
:1057A000281B01C020E0E1110BC0F601822F30E27E
:1057B000882319F031938150FBCFC20ED11C20E019
:1057C000992329F0D6019C93F60131966F01C60109
:1057D0000396E2FE0AC03EE4D6013C9341E41196F2
:1057E0004C93119712963C9306C03EE6F601308327
:1057F00041E641833283FC01322F40E2332309F436
:1058000042C041933150FACF82FF44C0911102C08F
:1058100083E001C084E0811718F4212F281B01C008
:1058200020E0E1110BC0F601822F30E2882319F04D
:1058300031938150FBCFC20ED11C20E0992329F077
:10584000D6019C93F60131966F01C6010396E2FEE4
:105850000BC039E4D6013C933EE411963C9311977A
:1058600036E412963C9307C039E6F60130833EE6F3
:10587000318336E63283FC01322F40E2332319F0C4
:1058800041933150FBCFFC01E20FF11D10828EEFEE
:105890009FEFB7C0F1E0911101C0F0E06F2F70E011
:1058A0001416150624F49A012F5F3F4F02C021E021
:1058B00030E0260F371FBB2029F06B2D70E06F5FA3
:1058C0007F4F02C060E070E0260F371F612F70E04D
:1058D000261737071CF4121B212F01C020E03E2D94
:1058E000387159F4D601322F60E2332319F06D93E9
:1058F0003150FBCFC20ED11C20E0FF2331F0D60186
:105900009C93B6016F5F7F4F6B01E1110BC0F601F5
:10591000922F30E3992319F031939150FBCFC20EAF
:10592000D11C20E09F2D940F3A81782F7071A72E03
:1059300084FF03C0313309F49150191624F49930CF
:1059400018F098E001C091E0E42F852F57FF02C0C6
:10595000E0E080E06E2F782FE0E0F0E0AEE29A2EFB
:105960003A01691A71082A01461A570A0B2D10E0EC
:105970001195019511096F3F8FEF780729F4D60132
:105980009C92C60101966C014617570784F0661673
:1059900077066CF47F01E40CF51CA1E0B0E0AC0FDD
:1059A000BD1FEA0EFB1ED7011196BC9002C090E30A
:1059B000B92E615071093196C60101967C016017BC
:1059C000710724F0D601BC926C01D5CF641775071E
:1059D00041F4363320F4353321F4A11002C081E3C1
:1059E000B82EF601B082F701822F90E2882319F0D9
:1059F00091938150FBCFF701E20FF11D108280E0FF
:105A000090E029960FB6F894DEBF0FBECDBFDF91B0
:105A1000CF911F910F91FF90EF90DF90CF90BF90AB
:105A2000AF909F907F906F905F904F900895A0E00F
:105A3000B0E0EDE1FDE20C94F230EC017B01611588
:105A4000710519F0DB018D939C938E010F5F1F4F41
:105A50007880872D90E00E94F62A892B11F0E801CA
:105A6000F4CFBDE27B1205C00F5F1F4F7980C1E00C
:105A700008C0EBE27E1204C08E010E5F1F4F7980DA
:105A8000C0E06801F1E0CF1AD10843E050E060E8DF
:105A900070E0C6010E944F2F892BF1F4680122E0CB
:105AA000C20ED11C45E050E06BE770E0C6010E94D9
:105AB0004F2F892B21F4680187E0C80ED11CE11417
:105AC000F10419F0D701CD92DC92C111FFC060E062
:105AD00070E080E89FE703C143E050E068E770E0D2
:105AE000C6010E944F2F892B51F4E114F10409F4EF
:105AF000F2C00E5F1F4FF70111830083ECC06801F5
:105B000060E070E0CB0100E010E0F601D0EDD70DD1
:105B1000DA3058F52C2F2260622E2C2F2870C2FF0D
:105B200005C0211128C00F5F1F4F25C0222311F08F
:105B300001501109A5E0B0E09B01AC010E94E330E7
:105B40004B015C01880C991CAA1CBB1CC501B4014B
:105B50006D0F711D811D911D6839A9E97A078A07AA
:105B6000A9E19A0740F0C66005C0DE3F51F4C3FDCD
:105B700044C0C8606C2EBFEFCB1ADB0A7080C62D04
:105B8000C4CF2D2F2F7D2531C1F540814D3211F429
:105B9000C06106C04B3221F0319621E030E006C0F2
:105BA0003296D60111964C9122E030E0A0EDA40F80
:105BB000AA3018F0E21BF30B20C040E050E0403860
:105BC000BCE05B075CF49A01220F331F220F331FE6
:105BD000420F531F440F551F4A0F511D3196DF01CD
:105BE00011972C91A0EDA20FAA3048F3C4FF03C077
:105BF000519541955109040F151FC1FF07C0E114CC
:105C0000F10421F03197D701ED93FC930E947C2F92
:105C1000C370C33019F06B017C0106C06B017C01BD
:105C2000F7FAF094F7F8F09420E030E0A901C7010A
:105C3000B6010E94772F882309F445C017FF06C0DC
:105C4000119501951109C7E9D0E002C0CFEAD0E073
:105C50005E01B8E1AB1AB1084601BE2DAF2D90E24E
:105C6000E92EF12C0E151F0584F0FE0125913591CA
:105C700045915491B4018B2F9A2F0E94DD2F4B0137
:105C8000B82FA92F0E191F09EDCF2497F594E7948B
:105C9000CA15DB0539F76401EB2EFA2E8E2D880F1D
:105CA0008F2D881F8F3F49F020E030E0A901C70108
:105CB000B6010E94772F811106C082E290E0909396
:105CC000010780930007C701B60109C060E070E0DA
:105CD00080E89FEF04C060E070E080EC9FE7CDB704
:105CE000DEB7EEE00C940E31283008F027E03327C1
:105CF000DA01990F311D87FD9160009661057105EC
:105D000039F432602E5F3D9330E32A95E1F7089530
:105D10009F3F30F080387105610509F03C5F3C5FC2
:105D20003D93913008F08068911DDF93CF931F93CE
:105D30000F93FF92EF92192F987F9695E92F9695E2
:105D40009695E90FFF27E35FFE4F99273327EE244F
:105D5000FF24A701E70105900894079428F4360F63
:105D6000E71EF81E491F511D660F771F881F991FD8
:105D70000694A1F70590079428F4E70EF81E491F32
:105D8000561FC11D770F881F991F661F0694A1F724
:105D90000590079428F4F80E491F561FC71FD11D00
:105DA000880F991F661F771F0694A1F70590079427
:105DB00020F4490F561FC71FD81F990F661F771F62
:105DC000881F0694A9F784911095177041F0D69515
:105DD000C79557954795F794E7941A95C1F7E3EB64
:105DE000F0E0689415901591359165919591059025
:105DF0007FE27395E118F10A430B560BC90BD009EA
:105E0000C0F7E10CF11E431F561FC91FD01D7EF4C1
:105E1000703311F48A95E6CFE894015030F0080F02
:105E20000AF40027021708F4202F2395022F7A3353
:105E300028F079E37D932A95E9F710C07D932A95A0
:105E400089F6069497956795379517951794E118F5
:105E5000F10A430B560BC90BD00998F023957E919C
:105E600073957A3308F070E37C932013B8F77E9132
:105E700070617D9330F0839571E37D9370E32A9593
:105E8000E1F71124EF90FF900F911F91CF91DF91D7
:105E9000992787FD90950895992788270895FB01F4
:105EA000DC014150504088F08D9181341CF08B35DD
:105EB0000CF4805E659161341CF06B350CF4605E0F
:105EC000861B611171F3990B0895881BFCCFDC01CF
:105ED000FC01672F71917723E1F7329704C07C9121
:105EE0006D9370836291AE17BF07C8F308950E9447
:105EF000B92F08F481E00895E89409C097FB3EF4B7
:105F000090958095709561957F4F8F4F9F4F992306
:105F1000A9F0F92F96E9BB279395F6958795779584
:105F20006795B795F111F8CFFAF4BB0F11F460FF44
:105F30001BC06F5F7F4F8F4F9F4F16C0882311F09C
:105F400096E911C0772321F09EE8872F762F05C0B0
:105F5000662371F096E8862F70E060E02AF09A954B
:105F6000660F771F881FDAF7880F9695879597F940
:105F70000895990F0008550FAA0BE0E8FEEF1616DA
:105F80001706E807F907C0F012161306E407F5072D
:105F900098F0621B730B840B950B39F40A2661F0A1
:105FA000232B242B252B21F408950A2609F4A14044
:105FB000A6958FEF811D811D08950E94F02F0C94EE
:105FC00061300E94533038F00E945A3020F09523FF
:105FD00011F00C944A300C94503011240C949530EC
:105FE0000E94723070F3959FC1F3950F50E0551FDA
:105FF000629FF001729FBB27F00DB11D639FAA271E
:10600000F00DB11DAA1F649F6627B00DA11D661F6C
:10601000829F2227B00DA11D621F739FB00DA11D8D
:10602000621F839FA00D611D221F749F3327A00D47
:10603000611D231F849F600D211D822F762F6A2FE3
:1060400011249F5750409AF0F1F088234AF0EE0F48
:10605000FF1FBB1F661F771F881F91505040A9F775
:106060009E3F510580F00C944A300C9495305F3F70
:10607000E4F3983ED4F3869577956795B795F795B1
:10608000E7959F5FC1F7FE2B880F911D9695879529
:1060900097F9089597F99F6780E870E060E00895A8
:1060A0009FEF80EC089500240A9416161706180630
:1060B0000906089500240A9412161306140605060C
:1060C0000895092E0394000C11F4882352F0BB0F9D
:1060D00040F4BF2B11F460FF04C06F5F7F4F8F4F00
:1060E0009F4F089557FD9058440F551F59F05F3F3B
:1060F00071F04795880F97FB991F61F09F3F79F0EA
:1061000087950895121613061406551FF2CF46956B
:10611000F1DF08C0161617061806991FF1CF8695ED
:106120007105610508940895E894BB2766277727D1
:10613000CB0197F90895F999FECF92BD81BDF89AE8
:10614000992780B50895262FF999FECF1FBA92BDE1
:1061500081BD20BD0FB6F894FA9AF99A0FBE019648
:106160000895DB018F939F930E94E330BF91AF911D
:10617000A29F800D911DA39F900DB29F900D1124A1
:106180000895A1E21A2EAA1BBB1BFD010DC0AA1F78
:10619000BB1FEE1FFF1FA217B307E407F50720F090
:1061A000A21BB30BE40BF50B661F771F881F991F0B
:1061B0001A9469F760957095809590959B01AC0154
:1061C000BD01CF0108950E942531A59F900DB49F78
:1061D000900DA49F800D911D112408952F923F9240
:1061E0004F925F926F927F928F929F92AF92BF92E7
:1061F000CF92DF92EF92FF920F931F93CF93DF9393
:10620000CDB7DEB7CA1BDB0B0FB6F894DEBF0FBEEF
:10621000CDBF09942A88398848885F846E847D843C
:106220008C849B84AA84B984C884DF80EE80FD803E
:106230000C811B81AA81B981CE0FD11D0FB6F894B4
:10624000DEBF0FBECDBFED010895A29FB001B39F89
:10625000C001A39F700D811D1124911DB29F700D6F
:10626000811D1124911D08955058BB27AA270E9413
:106270004C310C9461300E94533038F00E945A30F7
:1062800020F039F49F3F19F426F40C9450300EF4AA
:10629000E095E7FB0C944A30E92F0E94723058F3E6
:1062A000BA17620773078407950720F079F4A6F5FB
:1062B0000C9494300EF4E0950B2EBA2FA02D0B0108
:1062C000B90190010C01CA01A0011124FF27591B3B
:1062D00099F0593F50F4503E68F11A16F040A22F41
:1062E000232F342F4427585FF3CF469537952795B2
:1062F000A795F0405395C9F77EF41F16BA0B620BB1
:10630000730B840BBAF09150A1F0FF0FBB1F661FF7
:10631000771F881FC2F70EC0BA0F621F731F841F3A
:1063200048F4879577956795B795F7959E3F08F060
:10633000B0CF9395880F08F09927EE0F9795879522
:1063400008950E94B5310C9461300E945A3058F083
:106350000E94533040F029F45F3F29F00C944A30FA
:1063600051110C9495300C9450300E94723068F3A7
:106370009923B1F3552391F3951B550BBB27AA27FE
:1063800062177307840738F09F5F5F4F220F331F38
:10639000441FAA1FA9F335D00E2E3AF0E0E832D000
:1063A00091505040E695001CCAF72BD0FE2F29D003
:1063B000660F771F881FBB1F261737074807AB07D5
:1063C000B0E809F0BB0B802DBF01FF2793585F4F4A
:1063D0003AF09E3F510578F00C944A300C94953079
:1063E0005F3FE4F3983ED4F3869577956795B7952C
:1063F000F7959F5FC9F7880F911D9695879597F937
:106400000895E1E0660F771F881FBB1F62177307AF
:106410008407BA0720F0621B730B840BBA0BEE1FC4
:1064200088F7E09508950E941A326894B1110C948F
:10643000953008950E947A3088F09F5798F0B92FD0
:106440009927B751B0F0E1F0660F771F881F991FA9
:106450001AF0BA95C9F714C0B13091F00E94943087
:10646000B1E008950C949430672F782F8827B85F97
:1064700039F0B93FCCF3869577956795B395D9F701
:106480003EF490958095709561957F4F8F4F9F4F0B
:1064900008950E94B92F08F48FEF08950E94B92F34
:1064A000880B990B0895EE0FFF1F0590F491E02DD6
:1064B000099481E090E0F8940C94A332911108952E
:1064C00081568A5108F4805285580895FB01DC01F9
:1064D00002C001900D9241505040D8F708956817BE
:1064E000790768F4FB01DC01E40FF51FA40FB51F69
:1064F00002C002900E9241505040D8F708950C947B
:106500006632DC0101C06D9341505040E0F70895C0
:10651000FB01DC010D900020E9F7119701900D922D
:106520000020E1F70895FB01DC018D9101908019B5
:106530000110D9F3990B0895FB01DC0101900D9234
:0A6540000020E1F70895F894FFCF62
:10654A00FF6B116B110101FFFFFFFFFFFF00044DFD
:10655A0051545404DEEDBAFEFEEA0A00000000AA15
:10656A001012184210F1107310511065100000003B
:10657A00004E042104FA02F902000000002503205B
:10658A0003FA02521FED1BD01B1C1C4F03EC0260C6
:10659A001C0404DA023903C802EF02000000009169
:1065AA0011000000003D183D00525354003A006E9D
:1065BA00616E00696E66006F7666000D0A005341CF
:1065CA00564500312E31004A756C20313820323060
:1065DA0031390030393A35363A333500496E766109
:1065EA006C696421002F0043504D004D41580054FE
:1065FA004F540041564700454C50004856560046F5
:10660A0041430074657374757365720074657374BD
:06661A00706173730000C3
:00000001FF
